:02000000362B9D
:1000080070082000A1007108A00080312100901E16
:100018008A282000901E8A28230019082000C6007C
:1000280023009D1C28281D1219082000C600230043
:100038001D16013020004407F0000030453DF10056
:100048007008C4007108C50023001D1D3C289D13BD
:100058009D17013020004407F0000030453DF100B5
:100068007008C4007108C500230019082000C600E4
:10007800200046080D3A03194A284308003C031D8E
:10008800472842087E3C031C4A2870280130C900D2
:100098000030CA004308003C031D542842087E3C37
:1000A80003185A280230C9000030CA0021009012F3
:1000B8008030F0002230F1002000420870078600EE
:1000C8004308713D870081014208C7004308C80002
:1000D800C201C301C6018A288030F0002230F10035
:1000E8004208700786004308713D87004608810072
:1000F8004208C7004308C80001304207F00000303A
:10010800433DF1007008C2007108C30020002108B7
:08011800F0002008F1000900CD
:10012000290050082000D700290051082000D800DD
:10013000290052082000D900290053082000DA00C5
:10014000290054082000D300290055082000D400BD
:10015000290056082000D500290057082000D600A5
:10016000290058082000CF00290059082000D0009D
:1001700029005A082000D10029005B082000D20085
:1001800029005C082000CB0029005D082000CC007D
:1001900029005E082000CD0029005F082000CE0065
:0201A000080055
:0E01A20055303C008F00AA308F000F1408006B
:1001B0002000F801F9011030FC00710DF80DF90D67
:1001C0007408F8027508031C750FF9020318EF286C
:1001D0007408F80775080318750FF9070310F00D78
:0801E000F10DFC0BDD28080005
:1001E80023009E18F9280000F42820006208230044
:0401F8009A00080061
:1001FC0023009E1803290000FE282000620823001B
:04020C009A0008004C
:1002100023009E1690309D002000901E132923007D
:080220001908F0000C29080088
:0E02280055303C008F00AA308F000F100800E8
:10023600553023009600AA30960095140000000061
:020246000800AE
:100248002000DF0105305F02031834295F085D07CD
:10025800860000305E3D870020308100DF0A2629B5
:100268005F085D07860000305E3D87008101DF037F
:100278005F085D07E00000305E3DE1000A30F400F1
:10028800F5015B08F0005C08F100D8207808F00060
:100298007908F1003030F0076008860061088700AF
:1002A800700881000A30F400F5015B08F0005C0872
:1002B800F100D8207008DB007108DC0000307106FE
:1002C800031D682900307006031D6B296D29DF03A3
:0402D8003C290800B5
:1002DC0020005B082300910020005C0823009200A2
:1002EC0015131514000000001308F0001408F10099
:0202FC000800F8
:1002FE0014213D00A50194010D309D0012309F0088
:10030E0010309E0011309C000E303C00A0000C30CE
:0C031E00A1003D00A5019401D1200800C1
:10032A000D302000E200FE200A302000E200FE200C
:02033A000800B9
:10033C000B082000DF008B132300151515139516E1
:10034C0020005B082300910020005C082300920031
:10035C002000E0011F3060020318D1295D088400E1
:10036C005E0885000008230093000131000894000A
:10037C0002302000DD070030DE3D1B21013011076B
:10038C00F0000030123DF1007008910071089200ED
:10039C002000E00AB0292300951220005D0884009B
:1003AC005E088500000823009300013100089400CA
:1003BC001B2115112000DF1BE5298B13E6298B1758
:0203CC00080027
:1003CE00FF302900D000FF30D1000030D2000030C5
:1003DE00D300FE30D4000030D5006230D60000309D
:1003EE00D700FF30D800FF30D9000030DA000030DF
:1003FE00DB00FF30DC00FF30DD000030DE000030BF
:08040E00DF0090200821080026
:1004160020005B0884005C0885000008F000700876
:100426000319212A5B0884005C0885000008E200A5
:10043600FE202000DB0A0319DC0A0B2A0630FD0029
:08044600FD0B232A0000080051
:10044E0012001E00F003031D272AF103031D272AA5
:02045E00080094
:100460002000DE015B0884005C0885000008DD00D8
:100470005D08003A03194A2A5D08E200F4202000D2
:10048000DE0A5E085B07840000305C3D85000008E2
:06049000DD00382A08001F
:1004960020005D0884005E0885000008F0007008F2
:1004A6000319682A5D0884005E0885000008F000CC
:1004B6005B0886005C08870070088100DB0A031968
:1004C600DC0ADD0A0319DE0A4B2A5B0886005C0893
:0604D6008700810108000F
:1004DC0020005B08F2005C08F3007208F00073085F
:1004EC00F100F20A0319F30A700884007108850000
:1004FC0000080319822A732A5B087202F0005C0858
:0E050C00733BF1000130F0020030F13B0800BB
:10051A000B082000DD008B135B08230091002000EC
:10052A005C08230092001513151615151B211511C9
:0E053A002000DD1BA22A8B13A32A8B170800BA
:100548002200961323008C01FF3021008C000C122E
:1005580022000C1223008D01FF3021008D002400A1
:100568008D0125000D160D178D128D13F030260004
:100578008D0027008D0123008E01DF3021008E00C1
:10058800223024008E0021008E148E12951308004C
:1005980020005C08F000F036F036F036F036A23075
:1005A800840087308500700884070318850A0008CE
:1005B800F0005D0886005E08870070088100013041
:1005C8005D07860000305E3D87000F305C05F00057
:1005D800A230840087308500700884070318850AD4
:1005E8000008F0007008810002305D0786000030C6
:1005F8005E3D87005B08F000F036F036F036F036E6
:10060800A230840087308500700884070318850AA3
:100618000008F0007008810003305D078600003094
:100628005E3D87000F305B05F000A2308400873004
:100638008500700884070318850A0008F000700810
:10064800810004305D07860000305E3D870081012F
:02065800080098
:10065A0021009901191799161916991599149801D3
:02066A00080086
:10066C00EC302000A2008630A300F030A4008530CE
:10067C00A5006930A6008630A700AB30A8008530F5
:10068C00A9009230AA008730AB003030AC00863025
:10069C00AD002730AE008730AF00C130B0008730DE
:1006AC00B100B230B2008730B300CF30B400873025
:1006BC00B5002D23A4227F212000BC01BD01803078
:1006CC003D06F00080307002031D6E2B06303C029C
:1006DC000318962B22008E120C120B30FB002630C6
:1006EC00FC005D30FD00FD0B792BFC0B792BFB0B1B
:1006FC00792B000000008E160C160B30FB002630F8
:10070C00FC005D30FD00FD0B892BFC0B892BFB0BDA
:10071C00892B000000002000BC0A0319BD0A652BC0
:10072C00A030BE000330BF0023009F15CF309B00CC
:10073C009C011E15E7210A302000DB008730DC000D
:10074C000B220B30FB002630FC005D30FD00FD0B56
:10075C00AD2BFC0BAD2BFB0BAD2B00000000952142
:10076C004D302000DB008730DC000B22BC01BD01CA
:10077C0080303D06F00080307002031DC72B043022
:10078C003C020318DF2B3C08F0003D08F100F0356B
:10079C00F10D2230700784000030713D8500000897
:1007AC00DB0001310008DC000B22BC0A0319BD0A76
:1007BC00BE2B1530FB004B30FC00BE30FD00FD0B9A
:1007CC00E52BFC0BE52BFB0BE52B000022008E161A
:1007DC0095218B1330302000DB002130DC003630CB
:1007EC00DD008530DE004B223030DB002130DC00B8
:1007FC006E227008B6007108B7009C30DB008630A2
:10080C00DC000B22F0018E18F00A7008303EE2007A
:10081C00F420952120008E18922C3B30DB00873081
:10082C00DC000B22BC01BD0180303D06F0008030A5
:10083C007002031D232C80303C0203183D2C8030A9
:10084C003C07DB001F303D3DDC008D220230FB00FD
:10085C000430FC00BA30FD00FD0B322CFC0B322CAA
:10086C00FB0B322C0000BC0A0319BD0A1A2C5F309A
:10087C00DB008730DC000B223030DB002130DC0069
:10088C0030229521CD302000DB008630DC000B229D
:10089C003608DB003708DC00A030DD000030DE005D
:1008AC0024212030E200F420A0302000DB000030B6
:1008BC00DC00302295212000BC01BD0137083D022F
:1008CC00031D6A2C36083C020318922C80303C071E
:1008DC00DB001F303D3DDC003030DD002130DE0020
:1008EC003C08F0003D08F100F035F10D7008DD0713
:1008FC007108DE3D9E210230FB000430FC00BA3052
:10090C00FD00FD0B872CFC0B872CFB0B872C0000B0
:10091C00BC0A0319BD0A642C7130DB008730DC0083
:10092C000B229030F0002030F1007008BA007108F2
:10093C00BB007008B8007108B900BC01BD013708D4
:10094C003D02031DAB2C36083C0203182D2D3C0830
:10095C00DB003D08DC00A030DD000030DE0024218F
:10096C00A030DB000030DC0030220930E200F42043
:10097C00803020003C07DB001F303D3DDC006E2149
:10098C0070082000C0007108C10080303D06F000E6
:10099C0080307002031DD42C18303C02031C062D31
:1009AC0080303D06F00080307002031DDF2C1A30C1
:1009BC003C020318062D4008DB004108DC00A03087
:1009CC00DD000030DE00CC22A030DB000030DC008B
:1009DC0030220930E200F42020004108F000003001
:1009EC00C11BFF30F1007008E200F4200930200038
:1009FC00E200F420FF3020004005E200F4201D2D21
:100A0C0020004008DB004108DC00A030DD00003095
:100A1C00DE00CC22A030DB000030DC0030220930BC
:100A2C00E200F420FF3020004005E200F420952184
:100A3C008230FC00DD30FD00FD0B222DFC0B222D45
:100A4C00000000002000BC0A0319BD0AA52C95214A
:100A5C0082302000DB008730DC000B22342D352D5A
:100A6C006134623463346434653420346634203445
:100A7C006734203468342034693420346A342034A8
:100A8C006B3420346C3420346D3420346E34203488
:100A9C006F34203470342034713420347234203468
:100AAC007334203474342034753420347634203448
:100ABC007734203478342034793420347A34203428
:100ACC00303431343234333434342034353420340B
:100ADC00363420343734203438342034393420340C
:100AEC0041342034423420344334203444342034D0
:100AFC0045342034463420344734203448342034B0
:100B0C00493420344A3420344B3420344C3420348F
:100B1C004D3420344E3420344F342034503420346F
:100B2C00513420345234203453342034543420344F
:100B3C00553420345634203457342034583420342F
:0A0B4C00593420345A3420340034A8
:100B5600203453346F34753472346334653420343E
:100B66003A3420345F343134363446343134363412
:100B7600313439345F3454344534533454345F3467
:100B86004834453446345F345A346F346E346534F1
:100B96005F34553441345234543431345F34523432
:100BA600423437345F34543458345F345234423428
:100BB60035345F34523458345F343234303432345E
:100BC60030345F34303434345F34303431342E349E
:0A0BD600633420340D340A34003477
:100BE00020344434693472346534633474346F347B
:100BF0007234793420343A34203443343A345C3417
:100C00005F344D3469346B3472346F3443345C3444
:100C10005F344D3465347334503472346F346A3415
:100C20006534743473345F344D3469346B347234E6
:100C30006F3443345C345F343134363446343134C9
:100C40003634313439345F345434453453345434C5
:100C50005F3448344534463420340D340A3400348B
:100C600020345434653472346D3469346E346134F4
:100C70006C34203470346F347534723420346434FE
:100C8000693461346C346F346734753465342034BE
:100C900065347434203456346934733475342034F4
:100CA00020346434653472346F3475346C34653494
:100CB0006D3465346E3474342034703472346F346F
:100CC0006734723461346D346D3465340D340A34F4
:020CD0000034EE
:100CD2002034503472346F346A34653474342034BE
:100CE2003A342034543454346534733474345F34B5
:100CF2004834453446345F34313436344634313442
:100D02003634313439345F34553441345234543406
:100D12005F3432343034323430345F34303434344B
:100D2200303431342E346D34633470347034693479
:060D32000D340A34003408
:100D3800203454346534733474342034483445349E
:100D48004634203446346C346134733468343A346D
:100D58000D340A34203453347434613474347534A3
:100D6800733420346F3466342034503469346E342C
:100D780020344834453446345F344534633472345F
:100D880069347434293420345234433431343D3492
:020D9800003425
:100D9A0020345434613469346C346C34653420340E
:100DAA005A346F346E3465342034E0342034653478
:100DBA0063347234693472346534203465346E3481
:0E0DCA00203448344534463420343A34003462
:100DD80020344D3469346B3472346F3463342034C6
:100DE80037342E3436342E343034203450344934A9
:100DF80043342034313436344634313436343134A3
:0C0E08003934203420340D340A34003416
:100E1400203449346E3469347434203455344134C4
:100E240052345434313420345234423437343D341F
:100E34005434583420345234423435343D345234EA
:0A0E4400583420340D340A34003411
:100E4E00203441346C3469346D3420343D342034D4
:100E5E0033342E343334203474346F3420343534F8
:080E6E0056340D340A3400343F
:100E760020344534723461347334653420347A3422
:100E86006F346E34653420344834453446340D347A
:040E96000A340034E6
:100E9A002034503472346534733465346E347434A7
:100EAA006134743469346F346E3420343A340D3416
:040EBA000A340034C2
:100EBE0020345734723469347434653420345A34DF
:100ECE006F346E34653420344834453446340D3432
:040EDE000A3400349E
:100EE2002034523465346134643420345A346F34DB
:100EF2006E34653420344834453446340D340A3473
:020F02000034B9
:100F04002034663469346E34203454346534733494
:100F1400743420344834453446340D340A340034AF
:100F2400203444344534563449344334453420342D
:100F34003A3420344E346F3420340D340A340034BF
:100F44003034313432343334343435343634373461
:100F540038343934413442344334443445344634E7
:100F64002034413475347434723465347334203429
:0E0F74003A3420344E346F340D340A340034D5
:100F8200203446344F34533443343D3420343134E6
:0C0F920036342E3430340D340A34003470
:040F9E0020340034C7
:020000040001F9
:06000E00E438831E1F3FD1
:00000001FF
